:020000040000FA
:10000000D0230020150200001D0200001F02000086
:100010002102000023020000250200000000000071
:1000200000000000000000000000000027020000A7
:1000300029020000000000002B0200002D02000039
:100040002F0200002F0200003D0C00002F020000D4
:100050002F0200002F0200002F0200002F020000DC
:10006000F90B00002F0200002F0200002F020000F9
:100070002F0200002F0200002F0200002F020000BC
:100080002F0200002F0200002F0200002F020000AC
:100090002F0200002F0200002F0200002F0200009C
:1000A0002F0200002F0200002F0200002F0200008C
:1000B0002F0200002F0200000000000000000000DE
:1000C0002F0200002F0200002F0200002F0200006C
:1000D0002F0200002F0200002F020000000000008D
:1000E0000000000000000000000000000000000010
:1000F0000000000000000000000000000000000000
:1001000000000000000000000000000000000000EF
:1001100000000000000000000000000000000000DF
:1001200000000000000000000000000000000000CF
:1001300000000000000000000000000000000000BF
:1001400000000000000000000000000000000000AF
:10015000000000000000000000000000000000009F
:10016000000000000000000000000000000000008F
:10017000000000000000000000000000000000007F
:10018000000000000000000000000000000000006F
:10019000000000000000000000000000000000005F
:1001A000000000000000000000000000000000004F
:1001B000000000000000000000000000000000003F
:1001C000000000000000000000000000000000002F
:1001D000000000000000000000000000000000001F
:1001E000000000000000000000000000000000000F
:1001F00000000000000000000000000000000000FF
:10020000DFF80CD000F07EF90048004775150000BB
:10021000D02300200648804706480047FEE7FEE757
:10022000FEE7FEE7FEE7FEE7FEE7FEE7FEE7FEE7A6
:10023000DD0800000102000040EA01039B0703D033
:1002400009E008C9121F08C0042AFAD203E011F815
:10025000013B00F8013B521EF9D270470FB400B5C4
:1002600089B00BA800906A4603480A9900F040F94B
:1002700009B05DF814FB0000500000202DE9FF5F7D
:100280001D464FF0FF3BD5E9014691465F464FF0D2
:100290000008A9697F1C01988847296A8246884717
:1002A0000028F6D1BAF1FF3F0CD024F4C064002E30
:1002B00019DD600614D5BAF12B0F09D0BAF12D0F54
:1002C0000ED103E0584604B0BDE8F09F44F48064CA
:1002D000A9697F1C01988847761E8246002E02DDA0
:1002E000BAF1300F03D0B9F1000F26D032E0A9697E
:1002F000761E44F400747F1C019888478246002EC5
:1003000005DDBAF1780F06D0BAF1580F03D0B9F174
:10031000000F10D01EE0B9F1000F02D0B9F1100F9C
:1003200018D1A969761E24F400747F1C01988847AF
:100330008246102002E0082000E00A20814609E001
:1003400008FB0908A969761E44F400747F1C019813
:1003500088478246002E05DD4946504600F0BAF82F
:100360000028EDDAE96901988847A00502D46FF00A
:100370000100A8E7E00725D1600613D5600502D586
:10038000C8F1000000E0404629680A1D2A6009689B
:10039000220501D5087015E0220701D5088011E07B
:1003A00008600FE02868011D29600068210502D55A
:1003B00080F8008006E0210702D5A0F8008001E067
:1003C000C0F8008038467EE72DE9FF5FD2E901A73B
:1003D0004FF00008916999461446DDF838B046465A
:1003E00001988847054659EA0B0005D009E0A16944
:1003F000761C019888470546216A284688470028C8
:10040000F5D1681C03D05FEACA7005D015E04FF043
:10041000FF3004B0BDE8F09F2068011D2160D0F8D6
:1004200000800AE05FEACA7001D108F8015BA169A7
:10043000761C7F1E019888470546002F1ADD681C30
:1004400018D0B9F1000F0DD0E81705EBD0604211BC
:1004500020F01F0059F822102A1A01209040014272
:10046000E0D107E0BBF1000FDCD1216A28468847C4
:100470000028D7D0E16901988847BBF1000F07D168
:10048000002E05DD5FEACA7002D1002188F8001055
:10049000A068B84203DDBBF1000F03D017B16FF0C5
:1004A0000100B6E73046B4E730B50B460146002000
:1004B0002022012409E021FA02F59D4205D303FA26
:1004C00002F5491B04FA02F52844151EA2F10102A7
:1004D000F1DC30BD3A2800D2303820F02002412A29
:1004E00001D3A2F13700884201D34FF0FF307047AB
:1004F000024B9361024BD36100F032B8411100000E
:1005000045050000064C074D06E0E06840F0010399
:1005100094E8070098471034AC42F6D3FFF774FE16
:10052000A0270000C0270000094910B508784C1C1E
:1005300018B1401E0870205C10BD00210720ABBE22
:10054000207010BD02490878421C0A7070470000F4
:100550005800002002681144137801601846704763
:10056000D1600449516104491162002111611146B1
:1005700000F00AB8550500007D050000C0B24FF438
:10058000F05100F097B900002DE9F34F8BB04FF018
:10059000000801F10C000C464FF0010B46460DF12E
:1005A000080A01906269012101989047051E2DD02B
:1005B000252D2CD0216A8847C0B16269012101989C
:1005C0009047216A88470028F7D1411E6269019847
:1005D000904700E0761CA1690B988847216A8847FC
:1005E0000028F7D1E1690B988847DBE7A1690B98F0
:1005F00088470746A84201D1761CD3E7E1690B98EA
:1006000088477F1C02D1B8F1000F6FD046E1002768
:1006100062693D463946019890472A2804D16269AB
:100620000121019890470125DFF884926269012138
:1006300001989047A0F130010A290AD24F45E5DC24
:1006400007EB870100EB4107303FDFD445F0100591
:10065000ECE7E90601D46FF000476C280AD04C287B
:1006600014D0682815D06A280DD074281CD07A2898
:100670001AD01DE062690121019890476C2802D0D0
:1006800045F0040514E045F002050DE045F02005B5
:100690000AE06269012101989047682802D045F07C
:1006A000080505E045F4006562690121019890475D
:1006B000C4E9015765283DD019DC58287AD00CDCF4
:1006C000452837D004DC252826D0412831D131E017
:1006D00046282FD047282CD12CE05B2877D06128E2
:1006E00028D063287CD0642823D15AE0D0E06F283A
:1006F00048D008DC66281DD067281BD0692821D087
:100700006E2816D127E0702845D0732868D0752848
:1007100047D078280DD14DE0A1690B988847054650
:1007200025283FF469AFE1690B9888476D1C3FF4B9
:100730006AAFB3E023466A466FF001000B99AFF34E
:1007400000809EE045F040006060A80723464FF01F
:10075000000236D43EE0E8077FF447AF2068011D71
:1007600021600068290501D506701BE7290701D51E
:10077000068017E7A90703D5F117C0E9006111E763
:1007800006600FE745F040006060A80723464FF081
:10079000080216D41EE040F60E0125EA0100606052
:1007A00016E045F040006060A80723464FF00A02BB
:1007B00007D40FE045F040006060A80708D5234645
:1007C00010226FF001000B99AFF3008059E007E0B1
:1007D000234610226FF001000B99FFF74FFD50E008
:1007E0004FF000094F464B46632802D05B2806D0E5
:1007F00040E0E80601D40120A06001273AE06269E8
:100800000121019890475E2805D14FF001096269E6
:10081000494601989047216939B900210A46534653
:1008200043F82120491C0829FADBB0B3216969B9D2
:10083000C11700EBD16253110AEB830122F01F02B2
:10084000821A01200B68904003430B60626901210A
:10085000019890475D28E8D1B9F1000F09D0002038
:10086000514651F82020D24341F82020401C08284E
:10087000F7DB02AB224600976FF001000B99FFF700
:10088000A3FD00280CDA401C08D1BBF1000F05D0F5
:100890004FF0FF300DB0BDE8F08FFFE74046F9E7BD
:1008A000E90701D108F1010806444FF0000B79E691
:1008B000CCCCCC0C7F2801D9002208E0064A02EB00
:1008C0005002C007127800D1120902F00F02012075
:1008D00090400840704700001C270000F0B5B54864
:1008E0000023021D0178101D01254FF080540629B8
:1008F0000BD11678360708D10678C6F30316032EF7
:1009000006D0042E04D0052E02D0062907D00EE012
:10091000B4F82463A84FC6F304263E6002E01678BC
:10092000360704D10678C6F30316032E02D0062933
:1009300004D00FE0A24FA14E7E670EE01678360776
:1009400008D10678C6F30316032E06D0042E04D071
:10095000052E02D0062907D00EE0D4F84462994F44
:10096000C6F342363E6002E01678360704D10678B8
:10097000C6F30316032E02D0062906D011E0924ECC
:10098000376827F0807737600EE01678360708D191
:100990000678C6F30316032E06D0042E04D0052EC7
:1009A00002D006290AD011E04FF08046C6F80C317B
:1009B000C6F81031834E361F336002E016783607D2
:1009C00004D10678C6F30316032E02D0062905D0FB
:1009D0000CE07C4F032664373E600AE01678360749
:1009E00004D10678C6F30316032E02D006290DD0D3
:1009F00014E0764F05263E60744E78363560734EAF
:100A0000083633603F263F1D3E6002E01678360709
:100A100004D10678C6F30316052E02D0062957D056
:100A200062E06B4E36686B4F3E60694E361D36682D
:100A30003F1D3E60664E083636683F1D3E60644E80
:100A40000C3636683F1D3E60614E103636683F1DDD
:100A50003E605F4E143636683F1D3E605C4E183671
:100A600036685C4F20373E60594E1C3636683F1D55
:100A70003E60574E203636683F1D3E60544E243649
:100A800036683F1D3E60524E283636683F1D3E6038
:100A90004F4E2C3636683F1D3E604D4E3036366820
:100AA0004C4F40373E604A4E343636683F1D3E60FC
:100AB000474E383636683F1D3E60454E3C363668F8
:100AC0003F1D3E60424E403636683F1D3E6002E0AC
:100AD0001678360708D10678C6F30316032E06D01B
:100AE000042E04D0052E02D0062907D019E0D4F830
:100AF0005812394A01F04F01116002E011780907DC
:100B00000FD10078C0F30310032803D0042801D0CC
:100B1000052806D131480168C90702D06FF00101EC
:100B20000160D4F83001062808D1D4F83401062831
:100B300004D12B48016841F4806101602248743877
:100B4000016841F470010160BFF34F8FBFF36F8FF5
:100B50004FF01021D1F80002002803DBD1F8040285
:100B6000002822DA1F4A15601F480468002CFCD0B8
:100B70001524C1F800420568002DFCD0C1F80442DC
:100B800001680029FCD0136001680029FCD0BFF384
:100B90004F8F0D48F0380168144A01F4E0611143A9
:100BA0000160BFF34F8F00BFFDE712491048086096
:100BB000F0BD0000E00F00F0403501400DF0ADBA8F
:100BC00000C007403C050040FCED00E0105600402E
:100BD0000404001020C50040E40E00400004004062
:100BE0003C17004004E5014000E401400400FA0520
:100BF0000090D0035400002010B50E4C20466279BE
:100C0000017900782AB10A460146607801F01AFBA2
:100C100001E001F0EFFA2079401CC0B22071E178C8
:100C2000884201D9A078207103490020C1F8400111
:100C300010BD000010000020008000400148006846
:100C400000470000240000200FB4054B10B503A995
:100C5000044A029800F018F810BC5DF814FB00007C
:100C6000791100004C00002002E008C8121F08C1E2
:100C7000002AFAD170477047002001E001C1121F1D
:100C8000002AFBD1704700002DE9FF4F8BB09A4638
:100C90000F460546002606E025280BD052460D9942
:100CA00090476D1C761C28780028F5D10FB030468F
:100CB000BDE8F08F0024A0460122604900E0044313
:100CC00015F8013F203B02FA03F00842F7D12878DB
:100CD0002E2817D115F8010F44F004042A280ED04D
:100CE0006FF02F022878A0F1300109290AD808EB0B
:100CF000880102EB410100EB01086D1CF2E757F897
:100D0000048B6D1C287869283ED006DC0028CDD0E5
:100D100063280BD0642804D136E0732810D07528DE
:100D20004BD052460D999047761C85E017F8040B7E
:100D30008DF8000000208DF80100E946012003E055
:100D400057F8049B4FF0FF3061074FF0000401D4C7
:100D50000AE0641C44450DDA8442FADB19F80410F9
:100D60000029F6D106E0641C8442FCDB19F804106B
:100D70000029F8D1264404E019F8010B52460D99D8
:100D80009047641EF8D257E001CF4FF00A0B0028BD
:100D900002DA40422D2102E0210504D52B218DF8F5
:100DA0002410012103E0E10705D02021F7E70DF130
:100DB000200908910CE00021F9E701CF4FF00A0B60
:100DC000F9E75946FFF770FB01F1300209F8012DF0
:100DD0000028F6D1ADEB090000F1200B600701D42B
:100DE0004FF00108D84502DDA8EB0B0000E0002021
:100DF0008046002406E009A85246005D0D99904700
:100E0000641C761C08988442F5DB04E030205246CE
:100E10000D999047761CB8F10001A8F10108F5DCA6
:100E200005E019F8010B52460D999047761CBBF16D
:100E30000001ABF1010BF4DC6D1C34E70928010063
:100E400072B609480068C00700D000BEBFF34F8FDC
:100E50000548E4380168054A01F4E0611143016086
:100E6000BFF34F8F00BFFDE7F0ED00E00400FA058F
:100E70000EB500210091CDE901106A4644F201004F
:100E8000FFF7DEFF0EBD10B58268C368934203D042
:100E900000F05FF9002010BD052010BD29B112B18E
:100EA000531E134203D0092070470E207047016083
:100EB000838000218160C1600846704710B5826858
:100EC000C3689A1A83889A4203D800F04CF900202C
:100ED00010BD042010BD000070B50A4E01460A483E
:100EE000B578FFF7D0FF04464DB10020B070711CFB
:100EF0000122C81D00F00AFD08B1FFF7B9FF204626
:100F000070BD00002C000020AC030020F0B5244E82
:100F100089B01F460D00044672603FD0A88829683A
:100F200082B22048FFF7BAFF002835D1A889A96806
:100F300082B21C481030FFF7B1FF00282CD12022CC
:100F400019496846FFF778F960690690207C00B17E
:100F500001208DF814008DF81C70607C00B10E200B
:100F60008DF81500E0680290A06803902068019059
:100F7000606800900A480D4A6946083000F092FC0B
:100F8000002809D1B0702068401C05D00449012216
:100F9000491CC81D00F0BAFC09B0F0BD0720FBE7F2
:100FA0002C000020AC030020FC260000C123000020
:100FB00010B501461048FFF781FF040019D10F4812
:100FC0000F4A0178515C19B1001D00F097FF02E053
:100FD0000C3000F07BFE60B9084907480839FFF77C
:100FE00052FF30B9054901220839044800F09EFC3F
:100FF0000446204610BD0000BC0300203400002041
:101000001800002000F002B800F008B872B60248DC
:101010000168491C016070474800002003490868C6
:10102000401E086000D162B67047000048000020F2
:101030002DE9F041064608680C46411C4FF0A047D8
:101040004FF0010506D005FA00F1C7F80815206831
:1010500000F0B2FC6068411C02D0002100F09AFC54
:101060003168A069C1F82405607D227D3168104394
:10107000C1F86C05D4E900123068C0F81425C0F836
:101080000C15207D012815D1A068411C02D000213B
:1010900000F080FCE068411C05D08540C7F8085589
:1010A000E06800F089FCD4E902123068C0F8082535
:1010B000C0F81015BDE8F0812DE9F041064608683A
:1010C0000C46411C4FF0A0474FF0010506D005FA31
:1010D00000F1C7F80815206800F078FC6068411C32
:1010E00002D0002100F05FFC3168A069C1F824053E
:1010F000607D217D32680843C2F86C05D4E9001296
:101100003068C0F80C15C0F81425207D012815D1D1
:10111000A068411C02D0002100F045FCE068411CA1
:1011200005D08540C7F80855E06800F04FFCD4E9C9
:1011300002123068C0F80825C0F81015BDE8F0812B
:1011400008B56846FFF7C8FE0528FAD09DF80000EC
:1011500008BD826883881A4003689A5C0A708168B7
:10116000491C81607047C26883881A40036899549B
:10117000C168491CC160704710B50446C0B2FFF792
:1011800017FF204610BD000070B501F083F8154927
:10119000086000200446050201F07CF8641C284326
:1011A000E4B2042CF7D30F49083908600D49082030
:1011B00010390860091D0C4808600A4900201031E8
:1011C00008600A4DFE205FF00004287001F062F80C
:1011D0002919641CE4B24870FE2CF7D3014820386A
:1011E000056070BD24150040FF0004035C02002070
:1011F00008B51348FFF728FD694612A0FFF72EF83F
:101200009DF800003038022811D89DF800100EA07B
:10121000FFF71AFD9DF800100D4831290CD0302938
:101220000CD0012101700BA0FFF70EFD08BD0721B6
:1012300005A0FFF709FDDFE70021F3E70221F1E751
:101240005C2700002563000025630D0A00000000F4
:10125000000000200D0A000008B51AA0FFF7F4FCFA
:10126000694628A0FEF7FAFF9DF8000030380728ED
:101270000FD89DF80000FFF79BFE9DF80010224854
:10128000303907291BD2DFE801F0080A10121416C2
:1012900018000720FFF78CFEE2E7042100E00021A0
:1012A00041701AA0FFF7D0FC08BDFC21F8E7F82137
:1012B000F6E7F421F4E7F021F2E7EC21F0E7D8219A
:1012C000EEE70000456E746572206F75747075747A
:1012D00020706F77657220282730273D2B342064DB
:1012E000426D2C202731273D302064426D2C2E2E5C
:1012F0002E2C2737273D2D33302064426D293A0D9F
:101300000A00000025630000000000200D0A000014
:1013100010B514A0FFF798FC15A0FFF795FC24A0CA
:10132000FFF792FC2BA0FFF78FFC30A0FFF78CFC9F
:1013300039A0FFF789FC3FA0FFF786FC43A0FFF729
:1013400083FC4AA0FFF780FC4EA0FFF77DFC59A06C
:10135000FFF77AFC5CA0FFF777FCBDE810405FA0C8
:10136000FFF772BC55736167653A0D0A0000000013
:10137000613A20456E7465722073746172742063E3
:1013800068616E6E656C20666F722073776565703C
:101390002F6368616E6E656C20666F7220636F6E7E
:1013A0007374616E7420636172726965720D0A00F4
:1013B000623A20456E74657220656E6420636861D0
:1013C0006E6E656C20666F722073776565700D0AAE
:1013D00000000000633A2053746172742054582056
:1013E000636172726965720D0A000000643A2045FB
:1013F0006E7465722074696D65206F6E206561631F
:1014000068206368616E6E656C2028316D732D39BC
:10141000396D73290D0A0000653A2043616E6365DA
:101420006C2073776565702F636172726965720DE8
:101430000A0000006D3A20456E7465722064617484
:101440006120726174650D0A000000006F3A20533C
:1014500074617274206D6F64756C6174656420547E
:101460005820636172726965720D0A00703A2045F6
:101470006E746572206F757470757420706F776507
:10148000720D0A00733A205072696E74206375728F
:1014900072656E742064656C61792C206368616E7E
:1014A0006E656C7320616E6420736F206F6E0D0A21
:1014B00000000000723A2053746172742052582068
:1014C00073776565700D0A00743A20537461727405
:1014D0002054582073776565700D0A00783A2053C0
:1014E0007461727420525820636172726965720D62
:1014F0000A00000070B50D46044600684FF488717C
:1015000000F084FA4FF49071206800F07FFA4FF4F5
:101510009271206800F07AFA4FF4A271206800F00E
:1015200075FA20681249C0F8041320686907000B97
:1015300040B2090E002806DA00F00F0000F1E020AA
:1015400080F8141D03E000F1E02080F8001420680A
:101550000121000B40B200F01F02914040098000C1
:1015600000F1E020C0F88012C0F8001170BD00004A
:10157000100302008CB00024724801272646076041
:1015800080042546C0F80041C0F80070D0F8001172
:101590000029FBD018226C4901A8FEF74DFE6B48CC
:1015A000CDE907076A4809904FF400700A900723B5
:1015B000684A07A901A8FFF7A9FC08B1FFF758FC82
:1015C00065A0FFF741FB4FF0E0214FF48070A84683
:1015D000C1F8000162B65D4DED1E07A961A0FEF7DE
:1015E0003DFE9DF81C00613818286DD2DFE800F040
:1015F0000C1D3133496C6C6A6C6C6C6C4D6C5055C5
:101600006C585D606C6C6C6557A0FFF71DFB4F4913
:1016100063A0491CFEF722FE6868502801D80146E5
:1016200026E060A0FFF710FBEEE767A0FFF70CFBDA
:1016300046495BA0491DFEF711FEA868502804DC4E
:101640006868002801DBA96812E056A0FFF7FCFAE1
:10165000EBE7012440E069A0FFF7F6FA3B4950A010
:101660000931FEF7FBFDE868401E632805D2E968F2
:101670006FA0FFF7E9FA344626E06FA0FFF7E4FA1F
:10168000E9E700F0D7FD00261EE0FFF7B1FDF2E725
:10169000022472A0FFF7D8FA2AE0FFF7DDFDEAE79F
:1016A000052474A0FFF7D0FA44E000F035FC0BE00D
:1016B000032473A0FFF7C8FA26E0042473A0FFF701
:1016C000C3FA2AE0FFF724FE062C86D2DFE804F0F6
:1016D0000304101C253280E7A87818B100F0AAFD99
:1016E00085F802802A792978687800F0ABFD1EE041
:1016F000A87818B100F09EFD85F802802A79297833
:10170000687800F05DFD12E0287B00902B7A2A7942
:101710002978687800F0AEFD12E0A87818B100F0E2
:1017200089FD85F802802979287800F063FD264636
:10173000002452E72B7B2A7A2979287800F06AFD69
:10174000AF70F4E700D00040DC260000030000206A
:101750005C000020AF230000524620546573740DD6
:101760000A00000025630000456E746572207374E2
:10177000617274206368616E6E656C202874776F87
:1017800020646563696D616C206469676974732C9A
:1017900020303020746F203830293A0D0A000000C4
:1017A000256400004368616E6E656C206D7573740E
:1017B000206265206265747765656E203020616EF9
:1017C000642038300D0A0000456E74657220656E25
:1017D00064206368616E6E656C202874776F206486
:1017E0006563696D616C206469676974732C20306E
:1017F0003020746F203830293A0D0A00456E746528
:10180000722064656C617920696E206D7320287484
:10181000776F20646563696D616C206469676974C2
:10182000732C20303120746F203939293A0D0A0089
:1018300025640D0A0000000044656C6179206D7517
:101840007374206265206265747765656E2031204F
:10185000616E642039390D0A000000005458206D73
:101860006F64756C6174656420636172726965721E
:101870000D0A000052582053776565700D0A00006C
:1018800054582053776565700D0A00005258206344
:101890006F6E7374616E7420636172726965720D2C
:1018A0000A000000F0B505460478154889B01646D0
:1018B00040F82420124A0869121DA2F1080742F8D4
:1018C0002400487F385520226846FEF7B5FC049472
:1018D0002878385C48B10EB10A4A00E00022694617
:1018E000281D00F00BFA09B0F0BD0EB1064A00E069
:1018F0000022694605F10C0000F0B6F8F3E700009D
:101900001C000020B92500006124000030B40378D9
:10191000054CE35C1BB130BC001D00F025BA30BCA7
:101920000C3000F00BB900001800002030B4037830
:10193000054CE35C1BB130BC001D00F097BA30BC15
:101940000C3000F071B900001800002070B541EAB9
:101950004201DDE904564FF0A04441EA830141EA27
:10196000052104EB800041EA0641C0F8001770BD74
:1019700070B541EA4201DDE904564FF0A04441EA66
:10198000830141EA052104EB800041EA0641C0F8E9
:10199000001770BD1CB500220B4600921146019243
:1019A000FFF7D4FF1CBD1CB500220B460092114668
:1019B0000192FFF7DDFF1CBD1CB5002100910B4615
:1019C000012201911146FFF7C1FF1CBD1CB500218A
:1019D00000910B46012201911146FFF7C9FF1CBD82
:1019E0004058002800D00120704708B5002242501E
:1019F0004058009008BDD0F80403084000D00120F2
:101A000070474058002800D00120704708B50022D8
:101A100042504058009008BD0121B1EB507F01D1E8
:101A2000012070470020704770B50D4600F0AAFBFA
:101A300004000FD00020FFF7E5FA207920B1002044
:101A4000FFF7E2FA112070BD01202560207100200F
:101A5000FFF7DAFA002070BD0149024800F018BD16
:101A60005C030020002000402DE9F041054600798C
:101A700016460F4600EB40012D4A01EBC00102EB78
:101A8000810494F82A1011B10820BDE8F081294999
:101A900051F820102868FFF7C7FF08B11120F4E7BC
:101AA00039462846FFF7C4FA66603869206030007E
:101AB0004FF001062FD03F7F4FF48E712868FFF75B
:101AC00094FF4FF4A2712868FFF78FFF28681A4926
:101AD000C0F8041328684FEA4711000B40B20028F1
:101AE00006DA00F00F0000F1E02080F8141D03E09A
:101AF00000F1E02080F800142868000B40B200F0EC
:101B00001F0206FA02F14009800000F1E020C0F84F
:101B10008012C0F8001128680421C0F800150020C8
:101B2000A061E06184F8290044F8140FA675ACE7C1
:101B30005C030020F4260000800002002DE9F05F25
:101B4000054600794FF4017600EB400303EBC0003B
:101B5000344B03EB80040020636813B12B68C3F897
:101B60000863A3694FF000096BB1E06938B16068A0
:101B700010B12868C0F804631120BDE8F09FE2614D
:101B80000120216105E0C4F82490A261E160C4F85D
:101B90001C9094F82910014302D1284600F0BAFBAA
:101BA00060680028286803D0C0F804630020E4E7D8
:101BB0004FF4A2763146FFF718FFB2464FF4927BFE
:101BC00059462868FFF70CFF06464FF484712868D1
:101BD000FFF706FF804651462868FFF701FF0746DA
:101BE00048EA07003043EBD056EA070007D1214608
:101BF000286800F05FFBA169606A8142E0D8C4F800
:101C000018900EB10320B8E70FB10F20B5E794F894
:101C1000291001200029296801D00860C6E7486022
:101C2000C4E700005C0300202DE9F0470546007979
:101C30000B4600EB400101EBC000234901EB80049F
:101C4000284600F043F810B11120BDE8F0874FF0AE
:101C50000008C4F82080A360626184F828804FF4F3
:101C60008E76474631462868FFF7BFFE28684FF05A
:101C70000109C0F808902146286800F07BFB6068E5
:101C800000BBD5F800A00EE094F8280008B10F279B
:101C900016E031465046FFF7A3FE0028F4D0214657
:101CA000504600F067FB216A60698142F1D33146FA
:101CB0002868FFF795FE0028F9D02868C0F80C9036
:101CC000C4F814803846C0E75C030020007900EBBC
:101CD000400101EBC000044901EB8000406900288D
:101CE00000D00120704700005C0300200149024839
:101CF00000F07ABC88030020002000402DE9F0416C
:101D00000546164600790F46154A00EBC00102EB66
:101D1000810494F8201011B10820BDE8F081114928
:101D200051F820102868FFF77FFE08B11120F4E772
:101D300039462846FFF7C0F96660386920601EB151
:101D4000397F2846FFF7D6FB28680821C0F8001520
:101D50000020A061E0610121606184F82010DCE7CF
:101D600088030020F82600002DE9F05F0446007982
:101D70000E4600EBC001DFF8F0A017460AEB810524
:101D80003046FFF749FEB0B168684FF000084FF4E5
:101D9000047910B12168C1F80893A8694FF0000BCD
:101DA00080B1E86948B1686810B12068C0F8049350
:101DB0001120BDE8F09F1020FBE7EF614FF0010814
:101DC0002E6102E0EE60C5E9067B00254FF48871C4
:101DD0002068FFF71BFE4FF4A2712068FFF716FE84
:101DE0002068C0F83465C0F838752068B8F1000F75
:101DF00012D0D0F8001241F02001C0F80012207972
:101E0000D04600EBC0010AEB8100406838B1206881
:101E1000C0F804932846CCE701210160EFE74FF4B6
:101E2000887A4FF4A27951462068FFF7EAFD074609
:101E300049462068FFF7E5FD06464FF49271206899
:101E4000FFF7DFFD014647EA06000843EBD02279A1
:101E500002EBC20308EB8302C2F818B001B10325FC
:101E6000002ED7D00F25D5E7880300202DE9F047B5
:101E700004460E460079204900EBC00001EB8005C6
:101E800017463046FFF7C8FD30B1204600F036F85F
:101E900020B11120BDE8F0871020FBE76F61AE6034
:101EA0004FF49076002731462068FFF7AFFD4FF4DE
:101EB000AC7841462068FFF7A9FD2068AA686969E7
:101EC000C0F84425C0F84815206801218160686881
:101ED00078B9B14649462068FFF793FD064641466A
:101EE0002068FFF78EFD0643F4D000B10F270020D5
:101EF00068613846CEE70000880300200079054974
:101F000000EBC00001EB80004069002800D00120F8
:101F1000704700008803002010B523A0FEF794FE50
:101F2000254C207828B1012812D0022804D123A002
:101F300000E02BA0FEF788FE6078F0282DD009DCA9
:101F400088B104280DD0D8282BD0EC280ED126E05B
:101F50002CA0EFE7F4281ED0F8281AD0FC2805D1D1
:101F600015E031A000E038A0FEF76EFE3EA06168EB
:101F7000FEF76AFE43A0A168FEF766FE48A0E1688E
:101F8000FEF762FEBDE810404CA0FEF75DBE4DA01E
:101F9000EAE754A0E8E75BA0E6E762A0E4E769A00F
:101FA000E2E770A0E0E70000506172616D65746562
:101FB00072733A0D0A000000000000204461746151
:101FC00020726174652E2E2E2E2E2E2E2E2E2E2E4B
:101FD0003A20323530204B6269742F730D0A0000AD
:101FE0004461746120726174652E2E2E2E2E2E2E69
:101FF0002E2E2E2E3A2031204D6269742F730D0A39
:10200000000000004461746120726174652E2E2E00
:102010002E2E2E2E2E2E2E2E3A2032204D62697418
:102020002F730D0A00000000545820506F7765721E
:102030002E2E2E2E2E2E2E2E2E2E2E2E3A202B34BF
:102040002064426D0D0A0000545820506F7765726D
:102050002E2E2E2E2E2E2E2E2E2E2E2E3A203020AE
:1020600064426D0D0A0000002853746172742920C7
:102070004368616E6E656C2E2E2E2E2E3A202564DE
:102080000D0A0000456E64204368616E6E656C2E1B
:102090002E2E2E2E2E2E2E2E3A2025640D0A0000D6
:1020A00054696D65206F6E206561636820636861A7
:1020B0006E6E656C3A2025640D0A0000206D730D6C
:1020C0000A000000545820506F7765722E2E2E2E75
:1020D0002E2E2E2E2E2E2E2E3A202D342064426DA2
:1020E0000D0A0000545820506F7765722E2E2E2E48
:1020F0002E2E2E2E2E2E2E2E3A202D382064426D7E
:102100000D0A0000545820506F7765722E2E2E2E27
:102110002E2E2E2E2E2E2E2E3A202D31322064429F
:102120006D0D0A00545820506F7765722E2E2E2E9A
:102130002E2E2E2E2E2E2E2E3A202D31362064427B
:102140006D0D0A00545820506F7765722E2E2E2E7A
:102150002E2E2E2E2E2E2E2E3A202D323020644260
:102160006D0D0A00545820506F7765722E2E2E2E5A
:102170002E2E2E2E2E2E2E2E3A202D33302064423F
:102180006D0D0A000349884201D1034870470020C1
:102190007047000000200040240000200748002174
:1021A000C0F80012C0F8101101220261D0F810210D
:1021B000002AFBD0C0F8101170470000001000404A
:1021C00070B514460D460646FFF7E8FFFEF7DCFF44
:1021D00006480721C0F8001205490E60091D0D6070
:1021E0000349091F0C600121016070BD001000400F
:1021F0000C15004010B50C46FFF7D0FF0348012135
:10220000C0F80012024A1460416010BD0010004086
:102210000815004030B4044605480470817001710F
:10222000C2700021417130BC184600F083B8000034
:1022300010000020024901204860FFF7AFBF0000F6
:102240000080004070B514460D460646FFF7A6FF15
:1022500006480121C0F80012054A1660121D1560DB
:10226000034A121F1460016070BD0000001000409E
:102270000C15004030B4064C029D60702170A270B5
:102280002271E37001206071284630BC00F052B822
:102290001000002005480021C0F80011D0F80011FE
:1022A0000029FBD0024800687047000000D00040C1
:1022B00008D5004070B5054688690C4600284FF4E3
:1022C000847128460AD0FFF790FBD5F81805626A9A
:1022D000E1688854606A401C606270BDFFF785FB4E
:1022E000D5F8180570BD1FB501238DF80030CDE974
:1022F0000121D0E90012684690471FBD1FB5012398
:102300008DF800308DF808100192D0E9001268466F
:1023100090471FBD10B5044600684FF49271FFF757
:1023200064FB4FF484712068FFF75FFB2068012194
:10233000016010BD0D4910B501224A60C1F80022AC
:102340000B4C002323600223241D2360084C04232C
:102350000C3423601304C1F804334FF47A7310FB78
:1023600003F0034B3C3318600A6010BD008000404E
:102370000485004070B50C4605464FF48E71FFF79A
:1023800034FB216AA068415C206A401C2062C5F8C9
:102390001C1570BD1FB500228DF8002002918168C8
:1023A00001914261D0E90012684690471FBD017853
:1023B000022901D0012902D14068FEF759BD7047BA
:1023C0007CB50178244D81B301290BD002292BD192
:1023D0008DF80010C068691C01900122C81DFFF72C
:1023E00095FA2EE0406801781C48FEF767FD1B4C0B
:1023F000012618B18DF80060019006E0A068E16840
:10240000814205D000208DF8000069686846884741
:10241000A068E168081AA188884207D80E490122FD
:10242000491CC81DFFF772FA7CBD01E0AE70FBE7E6
:102430000A4809491030FEF726FD30B103208DF817
:102440000000696868468847EEE70349012201F108
:102450000800FFF76BFAE7E72C000020AC03002030
:102460001FB50A4601788DF8001041680191017A84
:102470008DF80810C0680390044850F82210001F1F
:1024800050F82220684690471FBD00002000002021
:102490002DE9FF470C4605464FF40071FFF7ABFAF4
:1024A00001274FF40178002618B34FF4927949467A
:1024B0002846FFF795FAE0B149462846FFF795FA16
:1024C000C5F8088394F8290000B96F6002208DF8E0
:1024D0000000D5F88004C5F880040390A06902903C
:1024E000E0680190A661E661D4E900126846904771
:1024F00028E004212846FFF77EFA18B34FF48471D0
:102500002846FFF76DFAE8B121462846FFF7D2FECC
:10251000616AA069884215D1E06938B1E268616AF0
:10252000A0612069E6616662E06008E094F8290035
:1025300000B96F60C5F80883A661E268616A204649
:10254000FFF7D1FE4FF48E7841462846FFF748FA50
:1025500078B1206A6169884202D294F8280020B3D9
:1025600041462846FFF741FA616911B12046FFF75D
:1025700011FF4FF4A27841462846FFF731FA0028B0
:1025800018D041462846FFF730FA94F8290000B1E8
:102590002F60A06900280DD0A661E268616A04B0CE
:1025A0002046BDE8F047FFF79EBE21462846FFF7CC
:1025B000E1FEDEE7BDE8FF871FB50A4601788DF82A
:1025C000001041680191017A8DF80810C0680390ED
:1025D000044850F82210001F50F822206846904707
:1025E0001FBD0000200000202DE9FF410C464FF4E4
:1025F000927705463946FFF704FA0026C0B13946FE
:102600002846FFF703FA02208DF80000D5F8800471
:10261000C5F880040390D5F83C058DF80800E06803
:102620000190A661E661D4E900126846904723E074
:102630004FF4887739462846FFF7E3F9E0B1394689
:102640002846FFF7E3F9D5F83C15A069884213D175
:10265000E06960B1E268D5F8000220F02000C5F81A
:102660000002E069A0612069E661E06001E0A66126
:10267000E2682046FFF742FE4FF4A277394628462B
:10268000FFF7BFF960B139462846FFF7BFF9A069E7
:1026900030B1A661D5F83C152046E268FFF72EFE62
:1026A0004FF4907739462846FFF7ABF9002813D04E
:1026B00039462846FFF7AAF9606900280CD0D5F8FA
:1026C0004C058DF800608DF80800A06801906661E7
:1026D000D4E9001268469047BDE8FF810800000079
:1026E00006000000050000000700000000000000D8
:1026F00000E0D701591A0000ED1C0000FFFFFFFFAA
:10270000FFFFFFFFFFFFFFFFFFFFFFFF00000000D5
:10271000000000000000D60107010000DDDDDDDD66
:10272000DCBBBBDDDDDDDDDDDDDDDDDD9888888862
:102730008888888877777777778888888555555609
:102740006666666666666666666888888333333260
:1027500022222222222222222228888D456E74657E
:1027600072206461746120726174652028273027AB
:102770003D323530204B6269742F732C202731276E
:102780003D31204D6269742F7320616E64202732C1
:10279000273D32204D6269742F73293A0D0A0000DB
:1027A000C0270000000000205C000000680C000052
:1027B0001C2800005C00002074230000780C00003E
:1027C0000100000000000000500000000A000000AE
:1027D00000000000000000000000000000000000F9
:1027E00000000000000000000000000000000000E9
:1027F0000000000000000000002000400000000079
:102800000020004000000000000000000000000068
:0C281000000000000090D0030000000059
:0400000500000201F4
:00000001FF
